:04000000F6EF04F023
:1000080000C016F001C015F03A0147AB10D0390115
:1000180090AF0DD03A01479BBA88010E3A24006E82
:10002800000E3B20016E00C03AF001C03BF016C044
:0800380000F015C001F01100F9
:0E004000550E3A01BF6FAA0EBF6FBF9112009E
:0E004E00550E3A01BF6FAA0EBF6FBF811200A0
:0C005C00000E3D01F9BF010E006E120005
:04006800F9DF1200AA
:10006C000001B851170802E2006A0ED3B951000A18
:10007C00D8A4B1D0BB5301E0DDDF60D06000EBF25F
:10008C0000FAA5D06000EBF201FAA1D06000EBF20F
:10009C0002FA9DD06000EBF203FA99D06000EBF20B
:1000AC0004FA95D06000EBF205FA91D06000EBF207
:1000BC0006FA8DD06000EBF207FA89D06000EBF203
:1000CC0008FA85D06000EBF209FA81D06000EBF2FF
:1000DC000AFA7DD06000EBF20BFA79D06000EBF2FB
:1000EC000CFA75D06000EBF20DFA71D06000EBF2F7
:1000FC000EFA6DD06000EBF20FFA69D06000EBF2F3
:10010C0010FA65D06000EBF211FA61D06000EBF2EE
:10011C0012FA5DD06000EBF213FA59D06000EBF2EA
:10012C0014FA55D06000EBF215FA51D06000EBF2E6
:10013C0016FA4DD06000EBF217FA49D00001B85115
:10014C00000A9CE0B851010A9DE0B851020A9EE0F9
:10015C00B851030A9FE0B851040AA0E0B851050A4F
:10016C00A1E0B851060AA2E0B851070AA3E0B851C1
:10017C00080AA4E0B851090AA5E0B8510A0AA6E099
:10018C00B8510B0AA7E0B8510C0AA8E0B8510D0AF7
:10019C00A9E0B8510E0AAAE0B8510F0AABE0B85169
:1001AC00100AACE0B851110AADE0B851120AAEE039
:1001BC00B851130AAFE0B851140AB0E0B851150A9F
:1001CC00B1E0B851160AB2E0B851170AB3E0000119
:1001DC00BB5301E036DF0001B951010AD8A451D15B
:1001EC00BB5301E027DFA4D06000E3F2C0FA45D195
:1001FC006000E3F2C1FA41D16000E3F2C2FA3DD1F2
:10020C006000E3F2C3FA39D16000E3F2C4FA35D1ED
:10021C006000E3F2C5FA31D16000E3F2C6FA2DD1E9
:10022C006000E3F2C7FA29D16000E3F2C8FA25D1E5
:10023C006000E3F2C9FA21D16000E3F2CAFA1DD1E1
:10024C006000E3F2CBFA19D16000E3F2CCFA15D1DD
:10025C006000E3F2CDFA11D16000E3F2CEFA0DD1D9
:10026C006000E3F2CFFA09D16000E3F2D0FA05D1D5
:10027C006000E3F2D1FA01D16000E3F2D2FAFDD0D2
:10028C006000E3F2D3FAF9D06000E3F2D4FAF5D0CF
:10029C006000E3F2D5FAF1D06000E3F2D6FAEDD0CB
:1002AC006000E3F2D7FAE9D06000E3F2D8FAE5D0C7
:1002BC006000E3F2D9FAE1D06000E3F2DAFADDD0C3
:1002CC006000E3F2DBFAD9D06000E3F2DCFAD5D0BF
:1002DC006000E3F2DDFAD1D06000E3F2DEFACDD0BB
:1002EC006000E3F2DFFAC9D06000E3F2E0FAC5D0B7
:1002FC006000E3F2E1FAC1D06000E3F2E2FABDD0B3
:10030C006000E3F2E3FAB9D06000E3F2E4FAB5D0AE
:10031C006000E3F2E5FAB1D06000E3F2E6FAADD0AA
:10032C006000E3F2E8FAA9D06000E3F2E9FAA5D0A4
:10033C000001BA51000AD8B457D7BA51010AD8B43F
:10034C0057D7BA51020AD8B457D7BA51030AD8B4FE
:10035C0057D7BA51040AD8B457D7BA51050AD8B4EA
:10036C0057D7BA51060AD8B457D7BA51070AD8B4D6
:10037C0057D7BA51080AD8B457D7BA51090AD8B4C2
:10038C0057D7BA510A0AD8B457D7BA510B0AD8B4AE
:10039C0057D7BA510C0AD8B457D7BA510D0AD8B49A
:1003AC0057D7BA510E0AD8B457D7BA510F0AD8B486
:1003BC0057D7BA51100AD8B457D7BA51110AD8B472
:1003CC0057D7BA51120AD8B457D7BA51130AD8B45E
:1003DC0057D7BA51140AD8B457D7BA51150AD8B44A
:1003EC0057D7BA51160AD8B457D7BA51170AD8B436
:1003FC0057D7BA51180AD8B457D7BA51190AD8B422
:10040C0057D7BA511A0AD8B457D7BA511B0AD8B40D
:10041C0057D7BA511C0AD8B457D7BA511D0AD8B4F9
:10042C0057D7BA511E0AD8B457D7BA511F0AD8B4E5
:10043C0057D7BA51200AD8B457D7BA51210AD8B4D1
:10044C0057D7BA51220AD8B457D7BA51230AD8B4BD
:10045C0057D7BA51240AD8B457D7BA51250AD8B4A9
:10046C0057D7BA51260AD8B457D7BA51270AD8B495
:10047C0057D7BA51280AD8B457D70001BB5301E05B
:10048C00E0DDA8D00001B9B102D0C29001D0C28089
:10049C00F9D00001B9B102D0C29201D0C282F2D01F
:1004AC000001B9B102D0C29401D0C284EBD00001DA
:1004BC00B9B102D0C29601D0C286E4D00001B9B164
:1004CC0002D0C29801D0C288DDD00001B9B102D0EF
:1004DC00C29A01D0C28AD6D00001B9B102D0C29C56
:1004EC0001D0C28CCFD00001B9B102D0C29E01D0D4
:1004FC00C28EC8D00001B9B102D0C39001D0C38064
:10050C00C1D00001B9B102D0C39201D0C382BAD01C
:10051C000001B9B102D0C39401D0C384B3D000019F
:10052C00B9B102D0C39601D0C386ACD00001B9B129
:10053C0002D0C39801D0C388A5D00001B9B102D0B4
:10054C00C39A01D0C38A9ED00001B9B102D0C39C1A
:10055C0001D0C38C97D00001B9B102D0C39E01D099
:10056C00C38E90D00001B9B102D0C49001D0C48028
:10057C0089D00001B9B102D0C49201D0C48282D01A
:10058C000001B9B102D0C49401D0C4847BD0000165
:10059C00B9B102D0C49601D0C48674D00001B9B1EF
:1005AC0002D0C49801D0C4886DD00001B9B102D07A
:1005BC00C49A01D0C48A66D00001B9B102D0C49CDF
:1005CC0001D0C48C5FD00001B9B102D0C49E01D05F
:1005DC00C48E58D00001B851000AD8B453D7B851C2
:1005EC00010AD8B456D7B851020AD8B459D7B85161
:1005FC00030AD8B45CD7B851040AD8B45FD7B85141
:10060C00050AD8B462D7B851060AD8B465D7B85120
:10061C00070AD8B468D7B851080AD8B46BD7B85100
:10062C00090AD8B46ED7B8510A0AD8B471D7B851E0
:10063C000B0AD8B474D7B8510C0AD8B477D7B851C0
:10064C000D0AD8B47AD7B8510E0AD8B47DD7B851A0
:10065C000F0A81E0B851100A85E0B851110A89E0FF
:10066C00B851120A8DE0B851130A91E0B851140A2E
:10067C0095E0B851150A99E0B851160A9DE0B851A9
:0A068C00170AA1E0FF0E006E120035
:10069600E8DC005202E10000FBD76000D7F2EAFD79
:0206A600120040
:1006A800B5C0B8F0B6C0B9F0B7C0BAF0010E0001D5
:0606B800BB6FD8DC12004C
:1006BE00A5C09AF0A6C09BF0A7C09CF0A8C09DF064
:1006CE00A9C046F0AAC047F0ABC048F0ACC049F094
:1006DE00ADC03EF0AEC03FF0AFC040F0B0C041F094
:1006EE00B1C042F0B2C043F0B3C044F0B4C045F064
:0206FE001200E8
:100700000001A5510308D8A0A56BA6510308D8A0E5
:10071000A66BF00E3D01F2170001A5513D01F21349
:10072000300EF213A6C000F00036009000360090A4
:1007300000360090003600900050F413F38F120042
:08074000A5C0B5F0A8DF12000E
:10074800086A096A100E0C6E01340836093604501E
:10075800085E0550D8A0053C095ED8B007D0045003
:1007680008260550D8B0053C0926D8900036013631
:060778000C2EEAD712006E
:10077E00160E0001B56FB66B130EB76F8EDF170E28
:10078E000001B56F010EB66F250EB76F86DF120032
:10079E00EFDFFF0E0001A56FFF0EA66F000EA76F15
:1007AE00000EA86F400EA96F070EAA6FA50EAB6FB5
:1007BE00000EAC6FFF0EAD6FFF0EAE6F000EAF6F83
:1007CE00000EB06F680EB16F000EB26F000EB36FF9
:0E07DE00000EB46F6DDFA56BA66B8BDF1200F3
:1007EC00520E0B6E2B0E0C6E000E0D6E0D2EFED7D8
:0C07FC000C2EFCD70B2EFAD700001200C8
:1008080009006F00D7FFE6FF0006FAE10106F8E1EC
:020818001200CC
:10081A003901DF87DF95DF93DF91DE6BDD6BD98DE1
:0E082A00D98BD999D997D995D993D991120024
:10083800CA6A020E3A01406FA30EC26E439DBA9671
:10084800506BCB6AC36AFF0E516F3E01BC6BB86B2D
:10085800CC6A3A01606B800EC46E3E01C16BC18FD9
:0A086800C183C1913A01636B1200D5
:100872000B6A0A6A096A005004026F00D0FF09F08D
:100882006F00CCFF08F0015005026F00D0FF0BF0A3
:100892006F00CCFF0AF000500502F3500926F45015
:1008A2000A22E86A0B2201500402F3500926F4508E
:1008B2000A22E86A0B2208C000F009C001F00AC04F
:0808C20002F00BC003F012006C
:1008CA0060007BF2F6FF60007FF2F7FF600083F2C0
:1008DA00F8FF09006F00D4FF00F0005215E0600035
:1008EA007BF2F6FF60007FF2F7FF600083F2F8FF09
:1008FA0009006F00D4FFA5F01EDF010E00019E273C
:0A090A00000E9F23A023DCD712008B
:100914000001A26B050EA25D0AE2A251A025E16EC0
:10092400000EA121E26E200EE66EA22BF3D7A25197
:10093400A025E16E000EA121E26EE66AA207A25193
:10094400A025A36F000EA121A46F0A0E046E000E51
:10095400056E9EC000F09FC001F0F4DE08C000F0F8
:1009640009C001F0300E002660008FF2E1FF600044
:1009740093F2E2FF600003F0E6FF0A0E046E000E3D
:10098400056E9EC000F09FC001F0DCDE00C09EF04A
:1009940001C09FF0000E011802E1000E001801E1F1
:0809A40002D0A207CCD712001B
:1009AC000D0E0001A56FC6DE0A0E0001A56FC2DE9A
:0209BC00120027
:1009BE0060007BF2E9FF60007FF2EAFFEE520EE08C
:1009CE0060007BF2E9FF60007FF2EAFF6F00B8FF84
:0E09DE00A5F0AFDE00019E4B9F2BEAD7120062
:1009EC000CEC07F014DF22DF386A396A000E395C30
:1009FC0002E1500E385C0AE24A0E3824E16E000E19
:100A0C003920E26EE66A384A392AF0D7BA8820ECE7
:100A1C0000F0130E166F170EE56F27EC00F0400E6A
:100A2C003D01F56F030EF66FF28FB3DEFF0E000182
:100A3C00A56FFF0EA66F000EA76F000EA86F400EDD
:100A4C00A96F070EAA6FA50EAB6F000EAC6FFF0E51
:100A5C00AD6FFF0EAE6F000EAF6F000EB06F680E75
:100A6C00B16F000EB26F000EB36F000EB46F21DECB
:100A7C00520E0B6E2B0E0C6E000E0D6E0D2EFED745
:100A8C000C2EFCD70B2EFAD700000C0EA56F52DEE5
:100A9C00FA0E00019E6F0D0E9F6F000EA06F0FDF00
:100AAC00386A396A000E395C02E1070E385C1CE2C8
:100ABC00030E006E000E016E38C004F039C005F054
:100ACC00D2DE170E0024E96E000E0120EA6E6F00D4
:100ADC00B8FF9EF06F00B8FF9FF06F00B8FFA0F05A
:100AEC00EEDE384A392ADED7BA983A6A3B6A3A01BE
:100AFC00448B476B458B469B3901A09F908FD28EC0
:100B0C003C6A3D6A3AC09EF03BC09FF04A0E000121
:100B1C00A06F000EA16FF8DE910E9E6F0D0E9F6FF1
:100B2C00000EA06FCCDE4A0E00019E6F000E9F6F70
:100B3C0040DF0F0E00019E6F0E0E9F6F000EA06F18
:100B4C00BEDE000ECABA010E0001A56F300EA5273D
:100B5C00F1DD090E0001A56FEDDDCAA81BD04B0E0F
:100B6C0000019E6F0D0E9F6F000EA06FA8DE3AC0A5
:100B7C009EF03BC09FF04A0E0001A06F000EA16FCB
:100B8C00C3DE4A0E9E6F000E9F6F13DF09DFBA980B
:100B9C003901908F05DF24DE3C4A3D2ACAD7FFD7A6
:100E180010EE17F0210E006E010E016E700EF66EC8
:0E0E28000D0EF76E000EF86E04EC04F01200D2
:020006002000D8
:100BAC0020436F6E66696720626974203A20503169
:100BBC00384632374B34325F466F73635F496E741D
:100BCC0065726E655F36344D687A5F776974685FFD
:100BDC005241365F436C6F636B6F75742E6366673F
:100BEC007363680D0A20464F53433A36342E302037
:060BFC004D487A0D0A00CD
:100C0200204469726563746F7279203A433A5C5F7B
:100C12004D696B726F435C5F4D657350726F6A65AD
:100C220074735F4D696B726F435C5F313846323764
:100C32004B34325F546573745F496E7465727275BA
:100C420070745F6F6E5F6368616E67655F52413596
:030C52000D0A0088
:100C550020557365206F6620612073706563696137
:100C65006C20616E74692D626F756E636520707599
:100C75006C73652067656E657261746F7220746F41
:100C850020646F206F6E6C79206F6E652070756CB7
:0D0C950073652061742074696D650D0A009F
:100CA20020536F75726365203A20504943313846AC
:100CB20032374B34325F55415254315F746573742D
:100CC2005F696E746572727570745F4F6E5F4368B0
:100CD200616E67655F5241355F5F323032315F303E
:080CE2003130352E630D0A00CC
:100CEA002050726F6A6574203A546573745F496E56
:100CFA00746572727570745F4F6E5F4368616E6778
:100D0A00655F31384632374B34325F323032312EFA
:080D1A006D637070690D0A00A1
:100D2200205465737420696E7465727275707420D4
:100D32004F6E204368616E6765206F6E20524135A9
:090D420020696E7075740D0A0041
:100D4B0020526973696E672045646765206F636322
:100D5B0075726564206F6E205241352020636F756C
:050D6B006E743D200044
:100D7000020C00E10D00EA0C00C70D00AC0B00AD49
:100D80000D00A20C00220D00550C00060000160EEE
:010D90000062
:100D910020526973696E67204564676520636F75CA
:0C0DA1006E74206F6E205241353D200022
:100DAD0020456570726F6D3A20206E6F74207573DB
:0A0DBD006564202E2E2E2E0D0A0074
:100DC70020546573742050494331384632374B34C9
:0A0DD700322020493243200D0A00AB
:100DE100204D696B726F432070726F20372E363041
:090DF1002042657461200D0A0026
:100DFA000D0A2050726573656E746174696F6E2096
:050E0A003A200D0A0072
:070E0F00205241353D200097
:020E16002000BA
:020000040030CA
:0A0000000428F5B70B3F9F0F010025
:00000001FF
